:020000040000FA
:0600000000008A11F52941
:08000800F200030E8301F10078
:100010000A088A01F000040883120313B9003908A2
:1000200083120313840070088A008301710E830019
:10003000F20E720E090083120313A701A801073004
:10004000A9000330AA00AD21CC2183120313B511FE
:100050009A214030392183120313B5159A21831256
:100060000313B5119A21C0303921003039210030F5
:100070003921003039210030392100303921003058
:100080003921003039210030392100303921003048
:100090003921003039210030392100303921003038
:1000A000392183120313B5159A2183120313B51155
:1000B0009A210330392183120313B5159A21831233
:1000C0000313B5119A214030392183120313B5155A
:1000D0009A2183120313B5119A21C030392183125A
:1000E0000313AA0300302A04031D7928A80A02304A
:1000F000AA00831203132808063A031D80288128CA
:10010000842883120313A801831203132808EF3EE7
:10011000AB0001300318013EAC002B08FE002C0898
:10012000FF0080308A11D2218A1183120313AD009F
:100130000F302705AB002B08E53EAB00013003185C
:10014000013EAC002B08FE002C08FF0080308A1115
:10015000D2218A1183120313AE00270E0F39AB0090
:100160002B08E53EAB0001300318013EAF002B0821
:10017000FE002F08FF0080308A11D2218A118312DD
:100180000313B000AB010730831203132B02031CCF
:10019000CA28FA280130831203133005AF00031078
:1001A0002F0DB1000310B10D01302E05AF0003106B
:1001B0002F0DB2000310B20D0310B20D3208B104BE
:1001C00001302D05AF002F0EF039B2000310B20D33
:1001D0000310B20D3208B104310839210030392141
:1001E000031083120313AD0C0310AE0C0310B00CFC
:1001F000AB0AC32883120313A90300302904031D8B
:100200000429A70A0730A9000F308312031327051A
:10021000AB002B080A3A031D0E290F2913290630BB
:1002200083120313A70783120313270E0F39AB00A2
:100230002B080A3A031D1D291E29212983120313A5
:10024000A70183120313B5159A216430FF00003013
:100250006E2183120313B5119A218F303921831235
:100260000313B5159A211030FF0027306E215F2847
:10027000080083120313A400A5010830831203139E
:100280002502031C44296A298312031335129A217B
:100290000130831203132405A6002608013A031D2A
:1002A0005229532957298316031387165E2983126F
:1002B0000313B5129A2183160313871203108312B6
:1002C0000313A40C8312031335169A21831203130C
:1002D000A50A3D298316031387160800831203130A
:1002E000A1007F08A000A201A3018312031321082B
:1002F0002302031D7D2920082202031C8029862950
:1003000083120313A20A0319A30A75290800831292
:100310000313050883120313B600831203130608A0
:1003200083120313B7008312031307088312031306
:10033000B8000800831203133308831203138500E7
:1003400083120313340883120313860083120313EA
:1003500035088312031387000800FF308316031348
:100360008500FF308600FF3087008312031385016C
:1003700086018701831203179E019F0183120313D5
:10038000B30183120313B40183120313B50183165F
:100390000313871107120800831603130F168F1615
:1003A0000F170800003A0319D929803A0319E029E8
:1003B00000347E08840083137F1883170008080028
:1003C0007F088A007E08820008003F3406345B34D0
:1003D0004F3466346D347D3407347F346F340234E7
:1003E000043410340834403420348A111B280800A7
:02400E00C43FAD
:00000001FF
